:100000000C942A000C945C010C945C010C945C012F
:100010000C945C010C945C010C945C010C945C01EC
:100020000C945C010C945C010C945C010C945C01DC
:100030000C945C010C945C010C945C010C945C01CC
:100040000C945C010C945C010C945C010C945C01BC
:100050000C945C0111241FBECFE5D8E0DEBFCDBFFC
:0C0060000E944E000C943400F894FFCF76
:10006C00424C494E4B494E47004C45465420534850
:10007C004946540052494748542053484946540075
:10008C00436C656172696E672053637265656E00BF
:10009C00CF93DF93CDB7DEB7E0970FB6F894DEBF02
:1000AC000FBECDBF8FEF81BB93E094BB8ABB17BA59
:1000BC002CE630E040E089E0F901DE011196742F66
:1000CC000E944F0125E730E040E08BE0F901DE01B2
:1000DC001A96742F0E944F0120E830E040E08CE02B
:1000EC00F901DE015596742F0E944F012CE830E087
:1000FC0040E080E1F901DE019196742F0E944F01DE
:10010C0088E30E94340180E80E9434018FE00E9451
:10011C00340186E00E94340181E00E943401B099E0
:10012C0020C081E00E943401CE0101960E94420160
:10013C008FEF8BBB2FEF40E782E021504040804097
:10014C00E1F700C000001BBA9FEF27E843E1915094
:10015C0020404040E1F700C0000081E00E943401E3
:10016C00DECFB1992AC081E00E943401CE010A96FB
:10017C000E94420180E88BBB8FEF90E722E0815018
:10018C0090402040E1F700C0000020E030E00EC0BD
:10019C008BB386958BBB4FEF80E792E0415080404C
:1001AC009040E1F700C000002F5F3F4F2830310531
:1001BC007CF381E00E943401B2CFB2992AC081E075
:1001CC000E943401CE0145960E94420181E08BBB16
:1001DC002FEF40E782E0215040408040E1F700C023
:1001EC00000020E030E00EC08BB3880F8BBB9FEF7C
:1001FC0040E782E0915040408040E1F700C00000B1
:10020C002F5F3F4F283031057CF381E00E94340191
:10021C0086CFB39984CF81E00E943401CE018196C0
:10022C000E9442019FEF29E648E191502040404056
:0E023C00E1F700C0000081E00E94340170CFA5
:10024A0082BB83E085BB2FEF80E792E0215080409C
:0E025A009040E1F700C0000081E085BB0895F0
:1002680082BB82E085BB2FEF80E792E0215080407F
:0C0278009040E1F700C0000015BA0895A6
:10028400CF93DF93EC0103C00E942501219688815E
:0A0294008111FACFDF91CF91089598
:10029E00992777FD05C005900D920197E1F7089516
:0A02AE0001900D920197E1F7089509
:0402B8000C940000A2
:00000001FF
